:10000000008000106D010000E1010000E701000028
:10001000ED010000F3010000F9010000F274FFEFB0
:10002000000000000000000000000000FF010000D0
:1000300005020000000000000B0200001102000099
:10004000170200001702000017020000170200004C
:10005000170200001702000017020000170200003C
:10006000170200001702000017020000170200002C
:10007000170200001702000017020000170200001C
:10008000170200001702000017020000170200000C
:1000900017020000170200001702000017020000FC
:1000A00017020000170200001702000017020000EC
:1000B00017020000170200001702000017020000DC
:1000C000170200001702000017020000D005000010
:1000D0000000001000000000D005000000C0072054
:1000E00000000000000000100400000000C0072015
:1000F0000000000080B489B000AFF860B9607A6099
:10010000BB68FB61FB68BB6100237B610AE0BA69E5
:10011000131DBB61FB69191DF96112681A607B69C7
:1001200004337B617A697B689A42F0D300BF24373D
:10013000BD4680BC704780B485B000AF7860396040
:100140007B68FB600023BB6007E0FB681A1DFA6058
:1001500000221A60BB680433BB60BA683B689A42ED
:10016000F3D300BF1437BD4680BC704780B584B060
:1001700000AF184BFB6013E0FB681A1DFA601B68A8
:100180003B60FB681A1DFA601B68BB60FB681A1DA8
:10019000FA601B687B607A68B9683868FFF7AAFF65
:1001A000FB680D4A9342E7D30DE0FB681A1DFA6025
:1001B0001B68BB60FB681A1DFA601B687B6079686E
:1001C000B868FFF7B8FFFB68044A9342EDD300F02C
:1001D000FDF9FEE7CC000000E4000000F4000000A0
:1001E00080B400AFFEE780B400AFFEE780B400AF9C
:1001F000FEE780B400AFFEE780B400AFFEE780B456
:1002000000AFFEE780B400AFFEE780B400AFFEE7CA
:1002100080B400AFFEE780B400AFFEE7FFFFFFFF52
:10022000FFFFFFFFFFFFFFFFFFFFFFFFFFFFFFFFDE
:10023000FFFFFFFFFFFFFFFFFFFFFFFFFFFFFFFFCE
:10024000FFFFFFFFFFFFFFFFFFFFFFFFFFFFFFFFBE
:10025000FFFFFFFFFFFFFFFFFFFFFFFFFFFFFFFFAE
:10026000FFFFFFFFFFFFFFFFFFFFFFFFFFFFFFFF9E
:10027000FFFFFFFFFFFFFFFFFFFFFFFFFFFFFFFF8E
:10028000FFFFFFFFFFFFFFFFFFFFFFFFFFFFFFFF7E
:10029000FFFFFFFFFFFFFFFFFFFFFFFFFFFFFFFF6E
:1002A000FFFFFFFFFFFFFFFFFFFFFFFFFFFFFFFF5E
:1002B000FFFFFFFFFFFFFFFFFFFFFFFFFFFFFFFF4E
:1002C000FFFFFFFFFFFFFFFFFFFFFFFFFFFFFFFF3E
:1002D000FFFFFFFFFFFFFFFFFFFFFFFFFFFFFFFF2E
:1002E000FFFFFFFFFFFFFFFFFFFFFFFFFFFFFFFF1E
:1002F000FFFFFFFFFFFFFFFFFFFFFFFFFFFFFFFF0E
:1003000080B500AF00F074F800F012F92E4B1B68B6
:100310002D4A43F0400313602C4B1B682B4A23F4F7
:10032000405313602A4B00221A602A4B63221A6042
:10033000294B44F620621A60284B4FF47A721A60F7
:10034000274B1B68264A43F002031360254B1B68AA
:10035000244A43F001031360224B1B68214A43F0F7
:10036000020313601A4B1B68194A43F400731360AD
:100370001D4B1B681C4A43F0020313601A4B1B6899
:10038000194A43F001031360174B1B68164A43F0E8
:1003900008031360154B4FF47A721A600EE0134B8A
:1003A0001A680E4B1A600F4B1B680E4A43F001038C
:1003B00013600E4B1B6801330C4A13600B4B1B6818
:1003C000B3F5FA6FEBDBE5E7C4C00F40A8C10F40FF
:1003D0004C8001400C800140188001401C8001408D
:1003E0001480014050800140048001400000001052
:1003F00080B400AF3C4B20221A6000BF3A4B1B6810
:1004000003F04003002BF9D0384B03221A60384B1D
:1004100000221A60374B00221A60374B01221A6003
:10042000364B374A1A60374BAA221A60354B552291
:100430001A60354B01221A60324BAA221A60314BE6
:1004400055221A6000BF314B1B6803F08063002BFC
:10045000F9D02D4B03221A602A4BAA221A60294B8D
:1004600055221A6000BF294B1B6803F04073002B14
:10047000F9D0274B23221A60264BAA221A60254B5B
:1004800055221A60244B01221A60224BAA221A60BC
:10049000204B55221A6000BF204B1B6803F4806379
:1004A000002BF9D01C4B03221A601A4BAA221A60A7
:1004B000184B55221A6000BF184B1B6803F4407399
:1004C000002BF9D0164B174A1A60174B00221A60FE
:1004D000164B1B6823F47043144A43F480431360A3
:1004E00000BFBD4680BC7047A0C10F4004C10F4093
:1004F000A8C10F40ACC10F400CC10F4084C00F40D9
:10050000630005008CC00F4080C00F4088C00F40C2
:10051000A4C00F40ACC00F40A0C00F40A8C00F4007
:10052000C4C00F40DE872804C8C10F4000C00F4080
:1005300080B500AF02220021022000F002F800BFC7
:1005400080BD80B483B000AF0346FB710B46BB7126
:1005500013467B71FB795B00DAB2BB791B09DBB216
:100560001344FB71BB7903F00F03DBB25B00BB717B
:10057000FB799B0003F1804303F530331A68BB79A4
:10058000032101FA03F3DB431946FB799B0003F1D6
:10059000804303F530330A401A60FB799B0003F176
:1005A000804303F530331A687979BB7901FA03F394
:1005B0001946FB799B0003F1804303F530330A436E
:1005C0001A6000BF0C37BD4680BC7047FFF798BE6D
:040000030000016D8B
:00000001FF
